:020000020000FC
:0400000009C068C00B
:0200080098C09E
:10000C0082C08DC097C0D4C10FEF07BB0FEF08BBE8
:10001C0008E304BB07E005BB0BEF01BB00E002BB30
:10002C000FE50DBF04E00EBF21E011243324662739
:10003C0077278827AA27BB27CC27DD2703E0202E8C
:10004C000FEF402E442755270FEFB02EF02E0FEB5D
:10005C00802E902EA02EC02ED02EE02E00270093A6
:10006C0060000093610000936400009365000FEF43
:10007C000093620000936300009366000093670096
:10008C000EEF009368000093690000936A000093E0
:10009C006B0004E003BF00E00FBD03E00EBD00E009
:1000AC000BBD00E10ABD00E009BD00E408BD04E0A1
:1000BC0005BD0DE509BF01E805BF00E40BBF00E875
:1000CC0008B978948895FECF000090B3947094157D
:1000DC0009F41895492E92FF07C06CB57DB56031B7
:1000EC00730580F034BC189564B5683058F03DBC8D
:1000FC003CBC603830F066247724552411248827C2
:10010C0001C0862F1895883048F092FD07C0660C08
:10011C00771C551C1394803208F06394189592FD4B
:10012C0005C00CD06624772455241124189501E8B9
:10013C0004BD18950FEF3DBC0CBD189508E11016C9
:10014C0009F401D008958301102702951027012F7F
:10015C00169516950127102F169501270170172D4E
:10016C0012951170101709F00895172D10955094D1
:10017C00569417955694179556941795569417951B
:10018C0056941795072D07701615500609F008950B
:10019C0073FC0BC0A3015770409368005093690027
:1001AC000FD0AB9AA0E7B7E10AC0A30157704093F8
:1001BC006A0050936B0080D0AC9AC0E7D7E10895E9
:1001CC0010916300009162004017510720F4509386
:1001DC00630040936200109161000091600004176D
:1001EC00150720F4509361004093600020FC04C07C
:1001FC00509163004091620021FC04C05091610059
:10020C00409160005E3F09F450C04F3F07E050073B
:10021C0008F044C0413000E0500708F438C088248E
:10022C009924AA24BB2411E0443F510718F0445FE1
:10023C00514007C004EF11E0041B150BA8010AE0A4
:10024C00B02E483E03E0500720F0485E5340B39474
:10025C00F8CF443600E0500720F044565040A394A9
:10026C00F8CF4A3018F04A509394FBCF042F10D19A
:10027C00802E092D0DD1902E0A2D0AD1A02E0B2DDA
:10028C00003011F005D101C00FEFB02E08950FEF23
:10029C00B02E07EF802E902EA02E08950FEFB02ECB
:1002AC000EEF802E902EA02E08950FEFB02E0FEB98
:1002BC00802E902EA02E089510916700009166005C
:1002CC004017510720F4509367004093660010913B
:1002DC006500009164000417150720F45093650025
:1002EC004093640020FC04C050916700409166006C
:1002FC0021FC04C050916500409164005E3F09F4FC
:10030C0050C04F3F07E0500708F044C0413000E0B8
:10031C00500708F438C0CC24DD24EE24FF2411E06F
:10032C00443F510718F0445F514007C004EF11E0FF
:10033C00041B150BA8010AE0F02E483E03E0500701
:10034C0020F0485E5340F394F8CF443600E0500759
:10035C0020F044565040E394F8CF4A3018F04A50FD
:10036C00D394FBCF042F94D0C02E0D2D91D0D02E32
:10037C000E2D8ED0E02E0F2D003011F089D001C043
:10038C000FEFF02E08950FEFF02E07EFC02ED02EAA
:10039C00E02E08950FEFF02E0EEFC02ED02EE02E93
:1003AC0008950FEFF02E0FEBC02ED02EE02E0895F7
:1003BC0009ED02BF2A9509F428E032BAAD98E9EEAE
:1003CC00F1E0E20FF31D099407C009C00DC010C085
:1003DC0012C014C018C01AC088BA909A1895092D6A
:1003EC000F7708BB919A1895A8BA939A1AD01895BA
:1003FC00B8BA949A1895C8BA959A18950D2D0F7786
:10040C0008BB969A1895E8BA979A1895F8BAAD9AC7
:10041C0001D01895119709F4AB98219709F4AC9871
:10042C000895112703B3037002111FEF202E003023
:10043C0091F01F3F79F4033059F4409168005091CA
:10044C006900D4DE40916A0050916B004BDF089537
:10045C00CDDE48DF08950027009360000093610013
:10046C0000936400009365000FEF0093620000930B
:10047C00630000936600009367000FEFB02EF02E20
:10048C000FEB802E902EA02EC02ED02EE02E089595
:10049C000B3008F00BE0F4E0EEEAE00FF31D0491F2
:0E04AC000895C0F9A4B0999282F88090BF869E
:00000001FF
